:10000000CE28B600841780048413A201201CA2000D
:100010003608A2060130A000A1010008360522061C
:10002000031D0800A00A0319A10F0D280800A5014F
:10003000A400B5172730A30010302A200330A300F6
:10004000E8302A20A30164302A20A3010A302A20A4
:1000500024083528A2002508A1002408A000AD200E
:100060002008031DB513B51B0800303EA600380854
:1000700084000930A70003104220A60CA70B3C28DF
:10008000031442288413B51D512800083604351D79
:1000900036068000841700083604031C36068000EC
:1000A0005C2800083604031C360635193606800025
:1000B0008417360980055C28350D0639A0006520B7
:1000C000A100A00A652000007F2800308A002008D7
:1000D00082070134903403343034003457340C3404
:1000E000F434A301A200FF30A207031CA307031CE2
:1000F000C9280330A100E5307F207328A101F63E16
:10010000A000A109031C8A28FE300000A0070318E4
:100110008528A0076400A10F8428000020189028DB
:100120002018922808000310A00DA10DFF3E03180F
:1001300093282008C928A2000530A800230821021E
:10014000031DA428220820020430031801300319DB
:1001500002302805031DFF30C9281030A600A50174
:10016000A401210DA40DA50D2208A4022308031C3F
:10017000230FA5020318C3282208A4072308031885
:10018000230FA5070310A00DA10DA60BB128200871
:10019000C9288313031383126400080083160430F4
:1001A0008500860183120610061186100330A30015
:1001B000E83072200614013071208614A001053049
:1001C0008400043001202008BA002108BB0006107A
:1001D00086103A08A0003B08A100A30100309B2034
:1001E0008A110A12031D10298A110A120630B8005A
:1001F0008030B6000630B5005030362061303620F1
:1002000073303620203036206430362027303620B8
:100210006530362063303620683036206F30362027
:100220003A08A0003B08A10002309620BA0021083D
:10023000BB00E830BA0703300318013EBB070630A5
:10024000B8008030B6000630B5003B08A5003A087B
:1002500018200D3036200730A300D0307220BA01AC
:08026000BB01DA28630032291A
:02400E00753DFE
:00000001FF
